:100B1C00EEEDEBE7DEDDDBD7BEBDBBB77E7D7B77D5
:040B2C00FEFDFBF7D8
:100B080009104E6F772054696D65000609000000D2
:030B1800000000DA
:100AA1007F017E007D017C000DBD00010CED647EA7
:0E0AB1004C70F50FBF00010EEF640B4E70E6A7
:010ABF002214
:0E0B3000D287C292D291D2902087FDC290222D
:100AF400120B30C292C2918F80D290E4FF0FBF05D7
:030B0400FCC290A0
:010B070022CB
:10099D00120A57E51B120AC0E51B75F00A84E5F033
:1009AD002430FF120AC77F3A120AC7E51C120AC08B
:1009BD00E51C75F00A84E5F02430FF120AC77F3A72
:1009CD00120AC7E51D120AC0E51D75F00A84E5F08F
:0609DD002430FF020AC7EE
:040A57007D077F0296
:100A5B00ED144480FEEF1475F040A42EFD120B3004
:100A6B00F580C292C291D290E4FF0FBF06FCC290F8
:010A7B002258
:070AC00075F00A842430FFE9
:100AC700120B308F80D292C291D290E4FF0FBF06F3
:030AD700FCC290CE
:010ADA0022F9
:100A7C008B208A218922AB20AA21A922120ADB60B1
:100A8C00130522E5227002052114F9120ADBFF126C
:050A9C000AC780E22200
:1009E3007F38120AF47F06120AF47F0C120AF47F8E
:1009F30001120AF47D017F01120A5B7F50120AC7BC
:100A03007D077F01120A5B7B007A007910120A7C52
:100A1300758901758CD8758AF0D2A9D2AFD28C8032
:010A2300FED4
:03000B00020800E8
:10080000C0E0C0F0C083C082C0D075D000C000C0BE
:0D08100001C002C003C004C005C006C0073F
:10081D00758CD8758AF0E519702C051EE51E64647B
:10082D007024051DE51DB43C17751D00051CE51C48
:10083D00B43C0D751C00051BE51BB41803751B009E
:10084D00751E0012099D0508E50864026003020883
:10085D00F6120A248F1FE50FF460030208F0E51F5E
:10086D00C394004039E51FD394095032E519640152
:10087D007071E51F2430FF120AC77408251AF8A6F7
:10088D001F051AE51A64036005E51AB405057F3ADC
:10089D00120AC7E51A6407704A120A578017E51F36
:1008AD00640A703FC3049519F519B4010D120A5766
:1008BD007F0F120AF4751A018029E50975F00AA453
:1008CD00250AF51BE50B75F00AA4250CF51CE50DA5
:1008DD0075F00AA4250EF51D7F0C120AF4751E0085
:0908ED0012099D750800851F0F1A
:1008F600D007D006D005D004D003D002D001D00056
:0B090600D0D0D082D083D0F0D0E032FF
:100A2400E4FE7DFFFCEC900B2C93F5A0AFA06F606F
:100A3400047E0180040CBC04ECBE0112E4FCEC90C6
:100A44000B1C93B50704AD0480040CBC10F0AE0578
:020A5400AF06EB
:010A5600227D
:03000000020911E1
:0C091100787FE4F6D8FD758122020958B9
:100ADB00BB010689828A83E0225002E722BBFE0219
:090AEB00E32289828A83E493224C
:10091D000209E3E493A3F8E493A34003F68001F204
:10092D0008DFF48029E493A3F85407240CC8C333DB
:10093D00C4540F4420C8834004F456800146F6DFAA
:10094D00E4800B0102040810204080900B08E47E27
:10095D00019360BCA3FF543F30E509541FFEE4939F
:10096D00A360010ECF54C025E060A840B8E493A366
:10097D00FAE493A3F8E493A3C8C582C8CAC583CA91
:10098D00F0A3C8C582C8CAC583CADFE9DEE780BE49
:010B1B0000D9
:00000001FF
